:020000040000FA
:1000000083160313CF308500C1308600813087000E
:100010008312031300309F008316031788008900A2
:10002000831203170730870088008316031370308C
:100030008F00F5309000243098000330990083122F
:10004000031390309800831603133030920083120C
:1000500003130C3092000C309B0020309D000130C7
:10006000900000308E008F000C10831603130C14C8
:1000700083120313003085000130860001308700B1
:100080000A168A11C9200A128A11B3019F24663008
:10009000B8000830B7243311851B752850306E0620
:1000A000031D752833156F08A0007008EE00710855
:1000B000EF007208F0007308F1007408F200750890
:1000C000F3007608F4007708F5007808F600790860
:1000D000F7007A08F8007B08F9002030FA00FB00EE
:1000E0006630B8000830DB247B2850306C06031DD6
:1000F00081286D08A0003130A00208302002031CC6
:1001000085282030EC00ED009A285030EC0031308A
:100110002007ED004C30B8002008B7244C08E6005A
:100120004D08E7004E08E8004F08E9005008EA00D3
:100130005108EB004C268830B9001130BA00B026C7
:1001400057269830B9001130BA00B0266226A9307F
:10015000B9001130BA00B0266D26B930B90011309F
:10016000BA00B02654245030A0004226E222B43017
:100170000F02031CB728A00BB52833107C2654248B
:10018000E22218232C25FF3A031DC028851B3311BA
:10019000E22218232C25FF3A0319C628FF3AB7009C
:1001A000331DD9280E303706031DBD280A128A15C3
:1001B0000028B708031DF32830306806031DF02817
:1001C00037306606031DE82836306706031907290D
:1001D000E7032F306706031DF0283930E700E603F8
:1001E0003030E8005B29013037060319FB28153051
:1001F0003706031D1E2937306606031D0E293630CB
:100200006706031D0E2930306806031D0E2939309C
:10021000E6003530E7003030E8001D29E8032F30D4
:100220006806031D1D293930E800E7032F306706F3
:10023000031D1D293930E700E6035B29023037062C
:100240000319262914303706031D4529393066065F
:10025000031D352935306706031D35293730E60083
:100260003630E7003030E8004429E80A3A306806C2
:10027000031D44293030E800E70A3A306706031DC1
:1002800044293030E700E60A5B2903303706031DB6
:100290005E293030E80039306606031D53293530B9
:1002A000670603192E29E70A3A306706031D5B2902
:1002B0003030E700E60AB31C9F24BD28043037061F
:1002C000031D66290030A00031309D290530370616
:1002D000031D6E290130A00032309D2906303706FB
:1002E000031D76290230A00033309D2907303706E0
:1002F000031D7E290330A00034309D2908303706C5
:10030000031D86290430A00035309D2909303706A9
:10031000031D8E290530A00036309D290A3037068E
:10032000031D96290630A00037309D290B30370673
:10033000031DB1290730A0003830ED005030EC002B
:100340004C30B8002008B7244C08E6004D08E70000
:100350004E08E8004F08E9005008EA005108EB0099
:10036000BD280C303706031DC0296A080925A000E6
:100370000C39EA00200A03396A041525EA00BD2871
:100380000D303706031DCE296B080925A000043067
:10039000A0070F3020051525EB00BD280E303706CD
:1003A000031DD329FD29103037060319DB2913302B
:1003B0003706031DE72950306C06031DE52931304F
:1003C0006D060319E5292E30F8290B30FB29113071
:1003D00037060319EF2912303706031DBD285030A8
:1003E0006C06031DFA2938306D060319FA292C30E2
:1003F0006D02FB290430B700D9283314B7017C26DD
:1004000018236226CB30B9001130BA00B0266D2611
:100410003708A000A00AA00B112AD630B90011306D
:10042000402AA00B172AE030B9001130402AA00B57
:100430001D2AF030B9001130402AA00B232A0530C4
:10044000B9001230402AA00B292A1530B900123009
:10045000402AA00B2F2A2730B9001230402AA00BC7
:10046000352A3630B9001230402AA00B3B2A4630DC
:10047000B9001230402AA00BFE295630B9001230C4
:10048000BA00B0262225A0000F302006031D492AFD
:10049000BD2814302006031D532AB70A0930370639
:1004A0000319B700FF2915302006031D5E2AB70384
:1004B000FF30370608300319B700FF290E30200639
:1004C000031D422A3708A0000319852A0A128A153B
:1004D000A00303190028A0030319082AA003031985
:1004E000BF2BA00303197B2CA0030319802DA003AD
:1004F0000319DC2DA0030319232E0A168A11A00369
:10050000031900280A128A11FE2950306C060030A7
:10051000031D8C2A31306D02A00062266630B900BE
:100520001230BA00B0266D266E30B9001230BA0013
:10053000B0267A26083020060A300319A02A200A9D
:10054000A1005430210792262225A1000F30210658
:10055000031DAB2AFF2914302106031DB52AA00A6A
:10056000093020060319A0009A2A15302106031D20
:10057000C02AA003FF30200608300319A0009A2AE1
:100580000E302106031DA42A083020060319DD2A97
:100590006608CC006708CD006808CE006908CF0067
:1005A0006A08D0006B08D1005030EC0031302007D1
:1005B000ED004C30B8002008E02A6630B800083062
:1005C000DB24BD2808266608E7256708E7256808B4
:1005D000E7256908E7256A08E7256B08E7250D3058
:1005E000E725EF25003A031D112B3F08C800EF2532
:1005F000003A031D112B3F08C900EF25003A031DE7
:10060000112B3F08CA00EF25003A031D112B3F08AC
:10061000CB00EF25003A031D112B0D303F060319C7
:1006200008004330C8003030C900CA00CB00102B8E
:10063000003092266C08E3266D08E3262030E3267E
:100640006608E3266708E3262E30E3266808E326DB
:100650004D30E3264830E3267A30E3262030E32687
:100660004808A201092501393130031D392BA20A9E
:100670002030E326220B412B30304906203003196D
:10068000422B4908E3264A08E3266430E326423039
:10069000E3262030E32648080925A200A218602B93
:1006A0002219662BA2195A2B0230E3265330E32677
:1006B00054306B2B0330E3264D30E3264E306B2B4A
:1006C0004F30E3265630E32646306B2B2D30E326A1
:1006D0002D30E3262D30E326403092265208E326C3
:1006E0005308E3265408E3265508E3265608E32674
:1006F0005708E3265808E3265908E3265A08E32654
:100700005B08E3265C08E3265D08E3265E08E32633
:100710005F08E3266008E3266108E3266208E32613
:100720006308E3266408E3266508E326143092266E
:100730006A0809250339A200A20AA20BAB2B733069
:10074000E3262E30E3267730E3266930E326643053
:10075000E3266530D22BA20BB92B7730E326693024
:10076000E3266430E3266530E3262030E32620309C
:10077000D22BA20BC72B6D30E3266930E326643001
:10078000E3266430E3266C30E3266530D22B6E30EE
:10079000E3266130E3267230E3267230E3266F30C1
:1007A000E3267730E3262030E3266B080925A200F4
:1007B000A219E02B6130E3267530E3267430E52B77
:1007C0006D30E3266F30E3266E30E3266F30E3268C
:1007D0002030E3266D30E3267530E3267430E326BF
:1007E0006530E3262D30E3266F30E3262219FC2BFB
:1007F0006E30E3262030FF2B6630E3266630E3269A
:100800006D26331D122C7030E3267230E3266F30D4
:10081000E3266730E3267230E3266130E3266D304D
:10082000E3262F2CB318212C6E30E3266F30E326FD
:100830007230E3266D30E3266130E3266C30E32628
:100840002F2C7330E3267030E3266530E3266330C7
:10085000E3266930E3266130E3266C30E32620305E
:10086000E3266B080925A200A21C3A2C3130E326AE
:1008700092303D2C9630221C4830C4266B30E32643
:100880004830E3267A30E3262030E3264C30E32656
:10089000690809250F39A2000A3022020030031826
:1008A00006302207C426080037306602031C842C59
:1008B0003A3066020318842C30306702031C842C03
:1008C0003A3067020318842C30306802031C842CF1
:1008D0003A3068020318842C37306602031D742CEA
:1008E00036306702031C842C39306602031D8B2CC2
:1008F000363067020318842C35306702031D8B2CB9
:100900003030680203198B2C3730E6003630E700B0
:100910003030E8009F24690809250F391525E900C2
:100920006A08092503391525EA006B0809250C39E1
:10093000EB007C0803396B041525EB000800203020
:10094000EC00ED00D200D300D400D500D600D700D3
:10095000D800D900DA00DB00DC00DD00DE00DF00BB
:10096000E000E100E200E300E400E5000800A2008E
:100970000310220DA200A300A20D220DA200A307C6
:10098000220D2307A200831203178D008313831205
:100990000313380884001A30A200831603170C14BE
:1009A000831203170C088D0A831203138000840A34
:1009B000A20BCD2C0800A2000310220DA200A30060
:1009C000A20D220DA200A307220D2307A20083126D
:1009D00003178D008D0383138312031338088400DB
:1009E0001A30A200831203130008840A831203172B
:1009F0008D0A8C00831603170C1555308D00AA3014
:100A00008D008C148C18022D83120313A20BF22C70
:100A10000800A4003030A4020A302402031C122D66
:100A20000730A4020F3024050800A4000F30A405ED
:100A30003030A4073A302402031C202D0730A407CD
:100A4000240808002C25FF3A031D222D2C25FF3AEF
:100A50000319262DFF3A0800831203138616063069
:100A6000A200A20B312D050886120F39BE000C30F2
:100A70003E18432D0D30BE18432D0E303E19432D28
:100A80000F30BE1D4E2DA2002430A400DB30A30089
:100A9000A30B482DA40B482D2208E62D33186C2DEE
:100AA0000D26003A031D6C2D12304406031D6C2DDB
:100AB00034304506031D6C2D46084707FF3A031DD9
:100AC0006C2DF0304605031D6C2D0E3046020030B3
:100AD000031802304607E62D86150630A200A20B49
:100AE0006F2DF030B4050F300505B4048611B51034
:100AF000351013303405013A031D812DB51235161A
:100B00003614361C8E2D03303405033A031D8E2D0A
:100B1000FC30B505350E0339B504361023303405E5
:100B2000023A031D962DB5163512B614B61CA32D28
:100B300003303405033A031DA32DFC30B505350EF3
:100B40000339B504B610CF30B405340E3039B404CF
:100B5000B51135114C303405043A031DB22DB513CF
:100B600035173615361DBF2D0C3034050C3A031DD4
:100B7000BF2DF330B505350E0C39B50436118C3068
:100B80003405083A031DC72DB5173513B615B61D24
:100B9000D42D0C3034050C3A031DD42DF330B5059B
:100BA000350E0C39B504B6113F30B405340EC039DA
:100BB000B40412303518E62D1330B518E62D143074
:100BC0003519E62D1530B519E62DFF3008008316CE
:100BD0000313981CE92D83120313990008000030B9
:100BE000BF008C1AF92DF42DF52DBF0BF12D03301C
:100BF000072E1819012E9818042E1A08BF0000306D
:100C0000072E1A080130072E181218160230080095
:100C10001A081A0818121816080001300718412E71
:100C20004226071C112E4226071C1C2E32300F02B2
:100C3000031C142E0630412E1D300F020330031CFE
:100C4000412E2030A500071C232E4226071C2E2EE5
:100C500016300F02031C262E0730412E08300F02DB
:100C6000C70DC60DC50DC40DA50B232E071C362EB2
:100C700042260530071C412E0E300F02031C392E70
:100C80000030080000308E008F000C108316031314
:100C90000C14831203130800003092261430A200B3
:100CA0002030E326A20B502E003092260800403060
:100CB00092261430A2002030E326A20B5B2E403097
:100CC00092260800143092261430A2002030E32629
:100CD000A20B662E1430922608005430922614304F
:100CE000A2002030E326A20B712E54309226080079
:100CF00018307D2E34307D2E3030A200C330870571
:100D0000051207080127C33087050512220887044A
:100D100001270530A3000A30A200A20B8D2EA30BE1
:100D20008D2E0800A400F039A5000310A50CA50C19
:100D3000A516C33087050512250887040127240856
:100D40000F39A5000310A50DA50DC33087050512A9
:100D50002508870401271830A500A50BAD2E080033
:100D6000C0260A128A11003A0319BF2EFF3A03194E
:100D7000BF2EFF3AE326B90A0319BA0AB02E0800BB
:100D80003A088A0039088200A200F039A300031053
:100D9000A30CA30CA30CA30C3030A3073A302302FE
:100DA000031CD42E0730A3070F30A2053030A20752
:100DB0003A302202031CDE2E0730A2072308E32666
:100DC0002208E3260800A4002408F039A500031037
:100DD000A50CA50CC3308705051625088704012737
:100DE00024080F39A5000310A50DA50DC3308705F4
:100DF00005162508870401271830A500A50BFE2E2F
:0E0E00000800851600008512C3308705080023
:10100000A030B80008300A128A11B7240A128A15D3
:10101000331D16280A128A116226A230B900123036
:10102000BA00B0266D260A128A152D280A128A11D6
:1010300057267F30B9001230BA00B02662266D26DE
:101040008D30B9001230BA00B026A0017A26831282
:10105000031314300A128A1192260A128A1550308C
:1010600083160313280683120313031D48288316CF
:1010700003132808831203130A128A11E326831626
:101080000313290883120313E3260A128A154E2834
:101090002A300A128A11E3262A30E32620300A1267
:1010A0008A11E3260A128A155030831603132A0682
:1010B00083120313031D6D28831603132A0883125A
:1010C00003130A128A11E326831603132B088312D3
:1010D0000313E3260A128A1573282A300A128A118A
:1010E000E3262A30E32620300A128A11E3260A1268
:1010F0008A155030831603132C0683120313031D25
:101100009228831603132C08831203130A128A11E0
:10111000E326831603132D0883120313E3260A1212
:101120008A1598282A300A128A11E3262A30E326E3
:1011300020300A128A11E3260A128A1550308316CB
:1011400003132E0683120313031DB72883160313FC
:101150002E08831203130A128A11E326831603133F
:101160002F0883120313E3260A128A15BD282A309A
:101170000A128A11E3262A30E32620300A128A1145
:10118000E3260A128A1550308316031330068312A1
:101190000313031DDC288316031330088312031383
:1011A0000A128A11E32683160313310883120313EC
:1011B000E3260A128A15E2282A300A128A11E32647
:1011C0002A30E32620300A128A11E3260A128A15F1
:1011D000503083160313320683120313031D0129B3
:1011E000831603133208831203130A128A11E326AB
:1011F00083160313330883120313E3260A128A1596
:1012000007292A300A128A11E3262A30E3262030E1
:101210000A128A11E3260A128A1550308316031324
:10122000340683120313031D26298316031334087F
:10123000831203130A128A11E32683160313350857
:1012400083120313E3260A128A1530292A300A1260
:101250008A11E3262A30E3260A128A153319412916
:10126000083020060A3003193B29093020061030C7
:1012700003193B29200AA100543021070A128A11C0
:1012800092260A128A1122250A128A15A1000F300D
:101290002106031D50290A128A11331DFF29BD287A
:1012A0003319412914302106031D5C29A00A0A3094
:1012B00020060319A000302915302106031D6729D7
:1012C000A003FF30200609300319A00030290E309A
:1012D0002106031D412908302002031C722903192D
:1012E000EF29012A83160313503028060319822997
:1012F0005030A800831203133130200783160313E4
:10130000A900272850302A06031990295030AA0036
:10131000831203133130200783160313AB002728F1
:1013200050302C0603199E295030AC008312031351
:101330003130200783160313AD00272850302E06C6
:101340000319AC295030AE0083120313313020074B
:1013500083160313AF002728503030060319BA292B
:101360005030B0008312031331302007831603136B
:10137000B1002728503032060319C8295030B20076
:10138000831203133130200783160313B300272879
:10139000503034060319D6295030B4008312031399
:1013A0003130200783160313B50027282A08A80028
:1013B0002B08A9002C08AA002D08AB002E08AC00B1
:1013C0002F08AD003008AE003108AF003208B00081
:1013D0003308B1003408B2003508B300CC298316B5
:1013E00003132030A800A900AA00AB00AC00AD0098
:1013F000AE00AF00B000B100B200B300B400B50061
:101400002728A030B80008300A128A11DB24BD2832
:10141000660883160313A00083120313670883165C
:101420000313A10083120313680883160313A20099
:1014300083120313690883160313A3008312031393
:101440006A0883160313A400831203136B08831620
:101450000313A50083120313520883160313A60077
:1014600083120313530883160313A7008312031375
:10147000540883160313A800831203135508831618
:101480000313A90083120313560883160313AA003B
:1014900083120313570883160313AB00831203133D
:1014A000580883160313AC008312031359088316DC
:1014B0000313AD00831203135A0883160313AE00FF
:1014C000831203135B0883160313AF008312031305
:1014D0005C0883160313B000831203135D088316A0
:1014E0000313B100831203135E0883160313B200C3
:1014F000831203135F0883160313B30083120313CD
:10150000600883160313B400831203136108831663
:101510000313B50083120313620883160313B60086
:1015200083120313630883160313B7008312031394
:10153000640883160313B800831203136508831627
:101540000313B900831203130A128A115726B2300B
:10155000B9001230BA00B02662268313A630840088
:101560001430A00000080A128A11E3260A128A1514
:10157000840AA00BB22ABB010A128A116D267A26B0
:101580000A128A15C32614303B070A128A119226C2
:101590000A128A15CB263D080A128A11E3263C0856
:1015A0007F39F83EA0000030031C6030A007BC1B50
:1015B000A017543092260A128A15AF23AF23AF2307
:1015C000AF23AF23AF23AF23AF2300300A128A111A
:1015D000E3260A128A15AF2301300A128A11E32684
:1015E0000A128A15AF23AF23AF23AF23AF23AF2354
:1015F000AF23AF23AF2314303B070A128A11922680
:101600000A128A1122250A128A15A1000F3021061A
:10161000031D0D2B0A128A11FF290C302106031D10
:10162000162BC3268030BC06CB26C02A15302106D7
:10163000031D232BBC0A3C087F39603A031D322B63
:101640008030BC05322B14302106031D342BBC0323
:101650003C087F397F3A031D322B3C088039803AA1
:101660005F38BC00CB26C02A12302106031D402B58
:10167000BB0A14303B06031DC02A0030BB00C02A41
:1016800013302106031D4C2BBB03FF303B06031D0B
:10169000C02A1330BB00C02A0E302106031D002BC8
:1016A0000A128A116D26C530B9001230BA00B02670
:1016B0000A128A1550306C060030031D612B313040
:1016C0006D02A0000A128A115530200792260A12D4
:1016D0008A1122250A128A15A1000F30210603194A
:1016E000BC2A14302106031D7B2BA00A08302006DB
:1016F0000319A000622B15302106031D862BA003C1
:10170000FF30200607300319A000622B0E3021069F
:10171000031D672BA030B80020080A128A11DB24B1
:101720000A128A1550306C060030031DAB2B4C306A
:10173000B80031306D020A128A11B7244C08E60055
:101740004D08E7004E08E8004F08E9005008EA009D
:101750005108EB00BD280A128A119F24BD282008D9
:10176000203E0A128A11E3260A128A15A00A2008CE
:101770007F39603A031DBE2B8030A0050800A00110
:101780000A128A116226CF30B9001230BA00B02690
:101790000A128A116D260A128A150030B900183013
:1017A000BA002008B9070318BA0A6E24A1006E24F3
:1017B000BA002108B9000A128A11B0260A128A1545
:1017C0006E240A128A1122250A128A15A1000F30EE
:1017D0002106031DEE2B0A128A11FF29143021065F
:1017E000031DF92B1E3020060319BF2B0230A00762
:1017F000C82B15302106031D062CA008031D032C41
:101800001E30A000C82B0230A002C82B0E302106CB
:10181000031DE12BA001A1014E24A10803191B2CDB
:10182000831603133730A0003630A1003030A200F9
:10183000831203133E2C6E2483160313A0006E2420
:1018400083160313A1006E2483160313A2008312D0
:1018500003138313A63084006E24A200A208031988
:101860003E2CFF30220603193D2CBA300406031922
:101870002C2C22088000840A2C2CA10AA030B8004D
:1018800020080A128A11DB240A128A15A00A0830DD
:101890002006031D0C2C0A128A11462883160313F6
:1018A0003330A3003130A4003030A5002030A60032
:1018B000A700A800A900AA00AB00AC00AD00AE00D4
:1018C000AF00B000B100B200B300B400B500B60084
:1018D000B700B800B9008312031308008312031382
:1018E00077240A128A15B90A0319BA0A08003A08B5
:1018F0008A0039088200A0010A128A1157260A12AA
:101900008A150030B9001830BA002008B90703184A
:10191000BA0A6E24A1006E24BA002108B9000A1286
:101920008A11B0260A128A156E243908C0003A08B6
:10193000C1003908C2003A08C3000A128A1162269F
:101940000A128A154208B9004308BA000A128A1519
:101950006E240A128A11E3260A128A156E240A12CC
:101960008A11E3262E30E3260A128A156E240A1203
:101970008A11E3262030E326B0264C26DD30B9005C
:101980001230BA00B0266D260A128A1122250A12D8
:101990008A15A1000F302106031DD12C0A128A11CD
:1019A000FF2912302106031DDC2C1E3020060319EE
:1019B0007B2C0230A0077C2C13302106031DE92C60
:1019C000A008031DE62C1E30A0007C2C0230A002D3
:1019D0007C2C14302106031DF92C4208B900430861
:1019E000BA006E24FF3A03199D2CFF3A031DF12C17
:1019F000992C15302106031D1B2D42084006031D9E
:101A0000052D4308410603199D2C4208B9004308DF
:101A1000BA00B903FF3039060319BA03B903FF301E
:101A200039060319BA0377240A128A15003A031DEE
:101A30000E2D6E24992C0E302106031DC42C0A1283
:101A40008A116D26C530B9001230BA00B026BC012B
:101A50007A260A128A1155303C0792260A128A11F8
:101A600022250A128A15A1000F30210603197A2DAA
:101A700014302106031D422DBC0A08303C06031910
:101A8000BC00292D15302106031D4D2DBC03FF3050
:101A90003C0607300319BC00292D0E302106031D1A
:101AA0002E2D4208B9004308BA004E246E24831636
:101AB0000313A0006E2483160313A1006E24831663
:101AC0000313A2008313A63084006E24FF3A031987
:101AD000722DFF3A0319722D8000840ABA30040275
:101AE000031C652D83120313A030B8003C080A12B2
:101AF0008A11DB240A128A117C260A128A159D2C6F
:101B00000A128A116226ED30B9001230BA00B026EE
:101B10006D260130B9001330BA00B0267A260A12B9
:101B20008A157C080339A000A0182010A0085530A1
:101B300003199F2D013020025B30031D61300A1212
:101B40008A1192260A128A1122250A128A15A100E8
:101B50000F302106031DAF2D0A128A11FF29143000
:101B60002106031DB92DA00A033020020319A0008D
:101B7000962D15302106031DC42DA003FF30200231
:101B800002300319A000962D0E302106031DA22D50
:101B9000A030B80008300A128A11B7242008FC00CF
:101BA00083160313B60083120313A030B800083065
:101BB000DB240A128A11BD280A128A116226153006
:101BC000B9001330BA00B0266D262A30B9001330A0
:101BD000BA00B026690809250F39A0000A128A1137
:101BE000553092260A3020020030031806302007B4
:101BF000C4260A128A1122250A128A15A1000F3062
:101C00002106031D062E0A128A11FF29143021060F
:101C1000031D102E0F3020060319F92DA00AEE2DFA
:101C200015302106031D192EA0080319F92DA00354
:101C3000EE2D0E302106031DF92D20080A128A11FF
:101C40001525E900BD280A128A1162263F30B90025
:101C50001330BA00B026A0010A128A116D260A12AA
:101C60008A152008A100A10AA10B3A2E5430B90010
:101C70001330912EA10B402E5E30B9001330912EFF
:101C8000A10B462E6730B9001330912EA10B4C2EBC
:101C90007030B9001330912EA10B522E7A30B9005A
:101CA0001330912EA10B582E8430B9001330912E91
:101CB000A10B5E2E8E30B9001330912EA10B642E35
:101CC0009830B9001330912EA10B6A2EA230B900C2
:101CD0001330912EA10B702EAC30B9001330912E21
:101CE000A10B762EB630B9001330912EA10B7C2EAD
:101CF000C030B9001330912EA10B822ECA30B9002A
:101D00001330912EA10B882ED630B9001330912EAE
:101D1000A10B8E2EE230B9001330912EF130B900B4
:101D20001330BA000A128A11B0260A128A1122252B
:101D30000A128A15A1000F302106031DA22E0A12D5
:101D40008A11FF2914302106031DAC2EA00A103081
:101D500020060319A0002C2E15302106031DB72ED6
:101D6000A003FF3020060F300319A0002C2E0E30E8
:101D70002106031D952E20080A168A11A6203A2056
:101D80000A128A15952E8313A6303B07840000089B
:101D9000E03EBC0008003C08203EBD008313A63096
:0A1DA0003B0784003D0880000800A6
:102000000A128A1162260030B9001430BA00B026D4
:102010006D260E30B9001430BA00B0267A26A00121
:10202000B318A00A5630201C5E300A128A1192267C
:102030000A128A1122250A168A11A1000F302106E0
:10204000031D25280A128A11FF29143021060319BD
:102050002D2815302106031D30280130A006122836
:102060000E302106031D1828B3102018B3140A12CD
:102070008A11BD2852202030A200C70DC60DC50D03
:10208000C40D03184528802046286920A20B3D284E
:1020900097204F30A300DE30A200A20B4D28A30BE7
:1020A0004D2808002C309D001630A5007D30A4007E
:1020B000A40B5828A50B582820309D00FD3087051B
:1020C0000B30A500BC30A400A40B6428A50B642829
:1020D00008002C309D000230A5005030A400A40B55
:1020E0006F28A50B6F2820309D00FD308705053037
:1020F000A5000830A400A40B7B28A50B7B280800B2
:102100002C309D000230A5005030A400A40B86287E
:10211000A50B862820309D00FD3087050230A500E4
:102120005030A400A40B9228A50B922808002C3054
:102130009D000230A5005030A400A40B9D28A50BE3
:102140009D2820309D00FD3087050800A400031065
:10215000A40DA40D2408483EA4001130A5000318C6
:10216000A50AC5200A168A11C400C2200A168A11BF
:10217000C500C2200A168A11C600C2200A168A119A
:10218000C7000800A40A0319A50A25088A00240824
:1021900082006030A3009F30A200A20BCD28A30BC9
:1021A000CD286400C330A2002208870505120C3038
:1021B000A200220887048516000085120A30A300B9
:1021C000D230A200A20BE228A30BE228C330A20067
:1021D0002208870505120C30A20022088704851604
:1021E000000085123D30A200A20BF428C330A200EB
:1021F0002208870505120C30A200220887048516E4
:10220000000085123D30A200A20B0429C330A200B9
:1022100022088705051287158516000085123D30B6
:10222000A200A20B1129C330A200220887050512C3
:102230008715851600008512C330A2002208870585
:10224000051287168516000085123D30A200A20BEC
:1022500027290A128A1178267C260A168A11C33089
:10226000870500000716051200008516000085127C
:1022700007128516000085121830A200A20B3E2915
:102280002030B9001430BA000A128A11B0260800B2
:10229000123434340034FF34123434340134FE3414
:1022A000123434340234FD34123434340334FC3404
:1022B000123434340434FB34123434340534FA34F4
:1022C000123434340634F934123434340734F834E4
:1022D000123434340834F734123434340934F634D4
:1022E000123434340A34F534123434340B34F434C4
:1022F000123434340C34F334123434340D34F234B4
:10230000123434340E34F134123434340F34F034A3
:102310002034543468346534203443344F344E34DC
:10232000543452344F344C344C34453452340034E9
:102330002034203466346F347234203446345034C0
:10234000473441342034743475346E346534723417
:102350000034203420342034203420346234793462
:1023600020346834693472346F346B3475346E34AD
:102370000034203420347634653472342E343234D0
:1023800030343134353430343234313434345F34F1
:102390007234653400347E344D34613469346E34C3
:1023A00020346D3465346E3475340034283431345F
:1023B00029345034723465347334653474340034E1
:1023C000283432342934503472346F3467347234E0
:1023D00061346D34203465346434693474340034C9
:1023E00028343334293453347434613474346934C4
:1023F0006F346E3420346E3461346D34653420347F
:102400006534643469347434003428343434293401
:10241000413472346534613420345234653471345B
:1024200075346534733474340034283435342934C5
:102430004134723465346134203443347534733438
:1024400074346F346D3469347A346534003428342C
:102450003634293453342F345034443449344634D8
:1024600020347234613474346534003428343734A1
:1024700029344F34753474347034753474342034E2
:102480004C346534763465346C3400342834383454
:102490002934533465346E3464342034493452342E
:1024A000203463346F346434653400342834393470
:1024B00029345334703465346334693461346C3492
:1024C00020346D346F346434653400347E345034D9
:1024D00072346534733465347434003450343134B8
:1024E00032343334343435343634373438342034B9
:1024F00049346E34693474345334543400347E3483
:10250000503472346F346734723461346D34203433
:1025100065346434693474340034503431343234C2
:102520003334343435343634373438342034433467
:102530006C3465346134723420345334613476340D
:10254000653400347E34503472346F3467347234FE
:1025500061346D34203473347434613474347534BC
:10256000733400347E3453347434613474346934D5
:102570006F346E3420346E3461346D3465342034FD
:102580006534643469347434003450343134323452
:1025900033343434353436343734383400347E34DC
:1025A00041347234653461342034523465347134CA
:1025B000753465347334743400347E344134723489
:1025C00065346134203443347534733474346F3477
:1025D0006D3469347A34653400347E3453342F34A6
:1025E00050344434493446342034733461346D34C7
:1025F00070346C346534203472346134743465342E
:1026000000342034343438346B3448347A34203451
:10261000393436346B3448347A34203431343934F4
:1026200032346B3448347A3400347E344F34753469
:10263000743470347534743420344C3465347634E6
:1026400065346C342034283430342D34313435340E
:102650002934003420343034333420342834533493
:10266000743461346E3464346134723464342034CC
:1026700069347334203430343334293400347E34B4
:10268000533465346E346434203449345234203445
:1026900063346F34643465342034283430342D345A
:1026A000313435342934003420342034303430345B
:1026B00020345B343C343C345D34003420342034EA
:1026C0003034313420345B343C345D3400342034D5
:1026D00020343034323420345B343E345D340034C2
:1026E000203420343034333420345B343E343E34B0
:1026F0005D340034203420343034343420345B34BE
:10270000503431345D3400342034203430343534A6
:1027100020345B34503432345D340034203420347F
:102720003034363420345B34503433345D34003448
:10273000203420343034373420345B345034343453
:102740005D340034203420343034383420345B3469
:10275000503435345D34003420342034303439344E
:1027600020345B34503436345D340034203420342B
:102770003134303420345B34503437345D340034F9
:10278000203420343134313420345B345034383404
:102790005D340034203420343134323420345B341E
:1027A0006D3465346E3475345D3400342034203437
:1027B0003134333420345B346234613463346B3409
:1027C0005D340034203420343134343420345B34EC
:1027D0005034723465347334653474342D345D345C
:1027E0000034203420343134353420345B345034D8
:1027F000723465347334653474342B345D3400348E
:102800007E345334703465346334693461346C34E9
:1028100020346D346F346434653400342034203413
:1028200045346E34613462346C3465342034203481
:10283000443469347334613462346C346534003444
:102840000F340E340C3408340C340E340F3480340E
:102850001E340E340634023406340E341E348034F2
:1028600011340A348034153480340A3411348034FD
:102870008034803404340E34043480348034803422
:02288000003422
:10300000203418344D3418347B341834BC3418341C
:10301000FB3418345F341934CA341934FE3419348B
:103020004A341A349C341A34E9341A3429341B349F
:1030300086341B34CA341B342F341C3466341C349D
:10304000303431342034CE34AF34B634B234C434B6
:10305000DE34B33400343834303434344134493419
:1030600052342D3447342734003438343234353434
:103070004E344F345234543448342034573441346D
:103080005634453400343834353432344E344834D0
:103090004B34203446344D34FF3430343234203411
:1030A000C434B334CE34B8342D34313400343734EE
:1030B0003634313446344D34203449345734413475
:1030C00054344534003438343034303441344634A8
:1030D00042340034383432343834413446344D3498
:1030E00000343834333431344E3448344B342034A3
:1030F00046344D34FF34303433342034C434B334A4
:10310000CE34B8342D34323400343734373431349B
:103110004434613474346534203466346D3400349E
:103120003834303434345234683479347434683454
:103130006D342034533474346134743469346F34EE
:103140006E340034383431343834463475346B34AA
:1031500075347334683469346D34613420344634E2
:103160004D3400343834323435344E3448344B34F2
:10317000203446344D34FF34303434342034B634C3
:10318000DD34C434B3342D34313400343734363480
:10319000343452344134443449344F34203442348A
:1031A0004534523452345934003437343834383496
:1031B00048346F3473346F342034443461346934A8
:1031C000673461346B34753400343834303433341C
:1031D0004E3448344B34203446344D340034383483
:1031E0003634333446344D342034473455344E3439
:1031F0004D344134FF34303435342034B634DD348A
:10320000C434B3342D3432340034373436343134AA
:1032100049346E3474346534723446344D34003479
:1032200037343834303462346134793466346D3450
:10323000003437343834363446344D342D34463443
:1032400055344A344934003437343934353446340B
:103250004D3420344E34413443344B34353400340F
:1032600038343034303454344F344B3459344F3490
:10327000203446344D3400343834313433344A3415
:103280002D345734413456344534003438343234D4
:1032900035344E3448344B34203446344D340034C5
:1032A00038343434373446346D34203479346F3420
:1032B0006B346F34683461346D346134FF343034CE
:1032C00036342034B634DD34C434B3342D3433349E
:1032D000003437343634313449346E347434653420
:1032E000723446344D34003437343934353446344E
:1032F0004D3420344E34413443344B34353400346F
:1033000038343034303454344F344B3459344F34EF
:10331000203446344D3400343834313433344A3474
:103320002D34573441345634453400343834353430
:1033300031344E3448344B34203446344D34003428
:1033400039343034353454344234533420345234E4
:103350004134443449344F34003439343134363410
:10336000423475346E346B346134203468346F34D5
:1033700073346F3400343934333430344E34693478
:10338000703470346F346E34203468346F34733476
:103390006F34FF34303437342034C134AD34B33477
:1033A000CC34DE3400343734393432344B342D34B9
:1033B0004D34493458340034373439343734463492
:1033C0004D342D344E344134473441344E344F342F
:1033D000003438343334303446344D342D344634AC
:1033E00055344A34493400343834353436344E3464
:1033F00048344B34203446344D34FF343034383480
:103400002034C434B334B634B234003437343734AF
:1034100038345A34493450342D3446344D34003421
:1034200037343834393472346134643469346F3445
:10343000203443345534423445340034373439343D
:10344000353449346E3474346534723446344D3412
:10345000003438343034303446344D34203447343A
:1034600049344634553400343834303437344634F3
:103470004D34203461346934633468346934003441
:103480003834323435344E3448344B3420344634B6
:103490004D34FF34303439342034CE34B834D83459
:1034A000B834003437343634313446344D34203473
:1034B000463455344B34553449340034373437347A
:1034C000353446344D342D344E3449344934473440
:1034D0004134543441340034373439343034463490
:1034E0004D34203450344F34523454340034383452
:1034F00030343534483445344C344C344F34203433
:103500004634493456344534003438343234323455
:103510004E3448344B34203446344D34003438343F
:103520003234373446344D34203454344F345934E3
:1035300041344D344134FF34313430342034B734E5
:10354000DD34B7342D343134003437343634353447
:1035500046344D34203443344F3443344F344C34A8
:103560004F34003438343034323446344D34383407
:1035700030343234003438343534313446344D3418
:1035800020344F34533441344B34413400343834D4
:10359000383431344E3448344B34203446344D348E
:1035A0000034383439343434E0342D345334543422
:1035B0004134543449344F344E340034383439347F
:1035C00039344B34693473347334203446344D34D5
:1035D000FF34313431342034B734DD34B7342D3452
:1035E0003234003437343734303465342D34723467
:1035F0006134643469346F340034383430343234F4
:1036000046344D3438343034323400343834353480
:10361000313446344D3420344F34533441344B34F8
:10362000413400343834373434344E3448344B3435
:10363000203446344D340034383439343434E034B2
:103640002D34533454344134543449344F344E348B
:10365000FF34313432342034C134AD34B334BA346D
:10366000DE34B834003437343634383446344D34EC
:1036700020344F344B344134593441344D34413487
:10368000003437343734343456342D3461346934AB
:1036900072340034373438343234483446344D349C
:1036A000003437343934323446344D3459340034EC
:1036B0003834383433344E3448344B342034463480
:1036C0004D3400343734373436344B346934733442
:1036D0007334203446344D3400343734383436347F
:1036E00046344D3420344B3441344734413457341C
:1036F0004134003437343934373446344D3420348F
:103700004534483449344D344534FF34313433344E
:103710002034BC34BA34B834003437343834363416
:1037200046344D3420344B344134473441345734DB
:103730004134003437343934373446344D3420344E
:103740004534483449344D34453400343834303409
:10375000373446344D34203454344F344B3455349C
:103760005334483449344D344134003438343134DE
:103770003634483469342D34533469347834003461
:103780003834373437344E3448344B3420344634AC
:103790004D34FF34313434342034B734AD34B334A1
:1037A000BC34AD34B3342D34313400343734363492
:1037B00031344C346F3476346534203446344D34EF
:1037C000003437343734343446344D344B340034D9
:1037D00037343734393446344D3453340034373485
:1037E00038343734633472346F3473347334203480
:1037F00066346D34003437343934353446344D341E
:1038000020344E34613467346134733461346B3442
:103810006934003438343034373446344D3420344D
:10382000463455344B3455344F344B3441340034E2
:103830003834343438344E3448344B3420344634FD
:103840004D340034383438343034413469347234CF
:10385000203452346134643469346F34FF34313489
:1038600035342034B734AD34B334BC34AD34B33430
:103870002D343234003437343734343446344D3414
:103880004B34003437343934383446344D342034F2
:103890006B34613467346F347334683469346D3435
:1038A000613400343834333432344A344F34593488
:1038B000203446344D3400343834353436344E34C4
:1038C00048344B34203446344D34FF3431343634AC
:1038D0002034B534B734C534DC34003438343734AC
:1038E000333466346D3420346F346B3469346E3461
:1038F00061347734613400343834383431344E3400
:1039000048344B34203446344D3400343834393460
:0A3910003134413446344E34FF34A4
:02400E00F42C90
:02401000FF3F70
:1042000037003600310033003100300049006E00C5
:1042100074006500720046004D0020002000200060
:10422000200020002000200020002000200020008E
:10423000200020003700380030003300310030000B
:1042400062006100790066006D00200020002000FF
:10425000200020002000200020002000200020005E
:1042600020002000200020003700380036003300F6
:104270003100300046004D002D00460055004A0038
:104280004900200020002000200020002000200005
:1042900020002000200020002000200037003900EE
:1042A000350033003100300046004D0020004E0044
:1042B000410043004B00350020002000200020007A
:1042C00020002000200020002000200020002000EE
:1042D00038003000300033003100300054004F000F
:1042E0004B0059004F00200046004D0020002000E8
:1042F00020002000200020002000200020002000BE
:10430000200020003800310033003300310030003D
:104310004A002D00570041005600450020002000B3
:10432000200020002000200020002000200020008D
:10433000200020002000200038003200350033002B
:10434000310030004E0048004B00200046004D0078
:10435000200020002000200020002000200020005D
:104360002000200020002000200020003800340021
:10437000370033003100300046006D002000790026
:104380006F006B006F00680061006D00610020002D
:10439000200020002000200020002000200020001D
:1043A000370036003100330031003000500031005A
:1043B00020002000200020002000200020002000FD
:0E43C00020002000200020002000200000002F
:00000001FF
